:020000040000FA
:0400000000003C2898
:080008008C108A015C083039FC
:100010008207510886005008831692008312103020
:04002000DC000900F7
:0E003200530886005208831692008312203075
:04004000DC000900D7
:0E005200550886005408831692008312003071
:04006000DC000900B7
:0E0072000030DC0009000230D0000030D10068
:100080006430D2008030D3009B30D4008030D50063
:10009000DC014130C000BD01C101C201C301C40186
:1000A000C501C601C701C801D8012030B8008312BC
:1000B000B901380884003908840783169B001C1492
:1000C0001A0883128000B90A0F303902031D59281B
:1000D0005A30B200B300B4003930B500B600323047
:1000E000B000B1012930B800B901BA01BB01BD01AE
:1000F00083160F308600831283160330920083121A
:100100000730920083164D309900203098008312FA
:10011000903098008B170B1783168C1483128B1753
:100120008C1A9528D81BD62A90288B131A08BC0045
:100130008C123B18EA28BA1BC42830088400310806
:10014000840700083C02031DAF28B10A05303102C4
:10015000031DB028B101B901FF30BA008F28B101E9
:10016000380884003908840700083C02031DC228AF
:10017000B90A05303902031D8F28B101B901FF30DA
:10018000BA008F28B9018F283C08BA00FF30BB00A5
:1001900000308A003A080F39D920CD004D080319E4
:1001A000F828BD01DA01CD1F8F28CD132808DA0009
:1001B0008F28820700340234823400340034003443
:1001C0000034003400340534013400340034003489
:1001D00000340034DA080319EF28DA038F284008C6
:1001E00084003D0884073C088000BD0ACD0B8F28A1
:1001F000BD01BB0101308A003A080F39023E0318E5
:100200008A0A82003C28122912293C283C283C28D2
:100210003C283C28962AA82A9E2A3C283C283C2890
:100220003C283C2801308A00420803391A3E031852
:100230008A0A820026292F2938299030DD004108BA
:100240008E21DF0041098E21DE004029A030DD0033
:1002500041098E21DF0041088E21DE0040296030F7
:10026000DD0041088E21DF0041098E21DE0040299A
:100270005030DD0041098E21DF0041088E21DE0073
:100280005F09031D5D295E08031D51290230D0005E
:100290006430D2009B30D400D101C030D300D500EF
:1002A00089290230D0005E08D200FF3CD400D10181
:1002B000F030D300C030D50089295E0903197029B8
:1002C0005E08D0005F08D4005F035E07D200D00252
:1002D000D4023030D100F030D300C030D5008929AD
:1002E0005F0803197F295F08D200FF3CD00002306D
:1002F000D4003030D100F030D300D50189296430EA
:10030000D0009B30D2000230D4003030D100D30076
:10031000D5015D08D105D305D5058F28E000013052
:100320008A006008963E03188A0A8200003402346C
:10033000033405340634083409340B340D340E34D8
:1003400010341134133414341634183419341B3463
:100350001C341E341F3421342234243426342734F0
:1003600029342A342C342D342F343034323433347D
:100370003534373438343A343B343D343E34403409
:100380004134433444344634473449344A344C3499
:100390004D344F3450345234533455345634583429
:1003A00059345B345C345E345F34603462346334BB
:1003B00065346634683469346B346C346D346F344E
:1003C00070347234733474347634773479347A34E4
:1003D0007B347D347E347F3481348234843485347C
:1003E0008634883489348A348C348D348E348F3416
:1003F00091349234933495349634973498349A34B3
:100400009B349C349D349F34A034A134A234A43452
:10041000A534A634A734A834A934AB34AC34AD34F5
:10042000AE34AF34B034B234B334B434B534B6349B
:10043000B734B834B934BA34BB34BC34BE34BF3446
:10044000C034C134C234C334C434C534C634C734F0
:10045000C834C934CA34CB34CB34CC34CD34CE34A4
:10046000CF34D034D134D234D334D434D534D53459
:10047000D634D734D834D934DA34DA34DB34DC3413
:10048000DD34DE34DE34DF34E034E134E134E234D0
:10049000E334E434E434E534E634E634E734E83491
:1004A000E834E934EA34EA34EB34EB34EC34ED3458
:1004B000ED34EE34EE34EF34EF34F034F134F13423
:1004C000F234F234F334F334F334F434F434F534F2
:1004D000F534F634F634F734F734F734F834F834C6
:1004E000F834F934F934F934FA34FA34FA34FB34A0
:1004F000FB34FB34FB34FC34FC34FC34FC34FD347E
:10050000FD34FD34FD34FD34FE34FE34FE34FE345F
:10051000FE34FE34FE34FF34FF34FF34FF34FF3446
:10052000FF34FF34FF34FF34FF34FF340830D7008A
:100530001130D9008130D800BA018F284108A800B5
:100540000830D7002830D6000130BE00BA01B92AE1
:100550004108A9004208AA004308AB004408AC00C7
:100560004508AD000930D7002930D6000530BE005F
:10057000BA0156088400000883169A0083125708AF
:1005800083169B009C111C1555309D00AA309D00C0
:100590009C141C1183128C1FCB2A8C13D70AD60AE9
:1005A000BE0BB92AB901BA01BB018F288B130C1EEF
:1005B0008F28570883169B001C141A088312990071
:0A05C000D70AD90B8F28D8018F2825
:02400E00613F10
:1042000000000000000000000000000000000000AE
:1042100000005600530049003900390020004100D9
:104220005200430052002000560031002E003000A2
:04423000300030002A
:00000001FF
